:100000000C94D1060C94F9060C94F9060C94F9069C
:100010000C94F9060C94F9060C94F9060C94F90664
:100020000C94F9060C94F9060C94F9060C94182615
:100030000C94F9060C94F9060C94F9060C94F90644
:100040000C942E2A0C94F9060C94F9060C94F906DB
:100050000C94F9060C94F9060C94F9060C94F90624
:100060000C9401290C94F906626F6F6D004765745A
:10007000206120626F6D6265004E6F206D61737448
:10008000657200536C61766520646973636F6E6E90
:1000900065637465640031206D6173746572206DF1
:1000A000617800536C6176652070617573656400DA
:1000B000507265737320616E79206B6579004024FE
:1000C0000000000000000000000000000000000030
:1000D000FF00000018000000FF00000018000000F2
:1000E000C0C3E60018000000C0C67A001800000077
:1000F000C0CE54F319E0FC67C0D9CCF319E0FC671B
:10010000FF11C6CCDE1B0378FF13FECCDE1B037889
:10011000C0DFFECCD81BFF60C0DFFECCD81BFF6069
:10012000C0CFFCCCDE1B0060C0C7F8CCDE1B00607B
:10013000FF03F0CCD9E0FC60FF01E0CCD9E0FC602B
:1001400000000000000000002060000000088004A3
:100150002090000004444F8823FC00000A22B9D0FC
:1001600024020000111109400801000024AA2130D6
:1001700029F90000494451180A950000920089F8B5
:100180000A950000494450F809F9000024AA20F813
:1001900004020000111300F00FFF00000A248FE09A
:1001A000130C8000044953C81294800000122004EC
:1001B0000F0F00000000000004F20000000000002B
:1001C000039C8000000001000000B29D1DDD9D0029
:1001D0007FFFB91111D149FE0000B11DDD5D49005D
:1001E000080570F870207058300000000000000012
:1001F0000000000060000000000000000000C09F40
:10020000C0000000000000007F20902000000000DF
:1002100000000081206017FFFFFFFFFFFFFD00C00F
:1002200020F60C104104100005E080215514975D64
:1002300055D5266550802154A59145551502255068
:100240008020F444974D75D66225E0801024A49454
:10025000451455222481000FC515D75D15D5777437
:100260007E000CC60C10410410000466000CC7FF91
:10027000FFFFFFFFFFFC66000B4404104104100069
:10028000045A000484E4104104100004240007050B
:10029000141041041000041C000005B410410410A7
:1002A00000040000800D5410410410000600204797
:1002B00095B41041041000051E402FC404104104E1
:1002C000100004BF000BE7FFFFFFFFFFFFFC2F80C4
:1002D00033F404104104100004CFC063F4E410416F
:1002E000041000058FC07E35B4104104100005F8DD
:1002F000C040351410410410000500C040255410C2
:10030000410410000500807224A41041041000056F
:10031000C8802514041041041000049440288FFF65
:10032000FFFFFFFFFFFCA220451404104104100052
:10033000051440A224E410410410000688801055E2
:1003400054104104100004414028CDF41041041021
:100350000004A3204525F4104104100005148088F2
:1003600094E41041041000062240104C0410410493
:10037000100004412028A7FFFFFFFFFFFFFCA28021
:1003800045140410410410000514400884E4104191
:1003900004100004220015455410410410000455B7
:1003A000002225F410410410000488804895F410C0
:1003B000410410000522402524E4104104100004EB
:1003C000948012440410410410000449000887FF7F
:1003D000FFFFFFFFFFFC22000500000000000000FF
:1003E00000140002000000000000000008000000EF
:1003F000000000000000000000581B00000000008A
:100400000000001100000008800030180CFF2222BC
:100410000004444F80381C0CC1D445000A22B84067
:10042000681C1CC0088880111100204C1E14C04597
:10043000524024AA20204C1A24C0A229204944500A
:1004400000C41A24FD10049092008800861B24C06A
:10045000A22920494451E1FE1944C045524024AA32
:100460002021821944C00C8880111300210319C473
:10047000C01245000A248023011884C0A922000468
:10048000495E62019884FF448000001221800000D0
:1004900000000000000008800400000000110000BF
:1004A00004444F8900DFE3F9A222000A22B9D18077
:1004B00090020A54450011110940819002040888F5
:1004C0008024AA2130C1900202455240494451186B
:1004D00041100202A22920920089F8431FE20D1068
:1004E0000490494450F8621003F8A2292024AA205D
:1004F000F826100230455240111300F03410021853
:100500000C88800A248FE01410020F124500044961
:1005100053C818100204A9220000122004081FE288
:1005200002448000080570A8F8F870080570D888A3
:10053000A85008057088D8A8D8010101010101015F
:10054000010101010101010101010101010101009C
:100550000000020200000000020202020202020089
:10056000000001010001020102010200020102017A
:100570000201020102010001010200020102010266
:100580000002010201020102010201020101020155
:10059000000000010200020102000201020002014B
:1005A0000201010201020002010201020102010234
:1005B0000002010201020101020002010200020127
:1005C0000201020102000201020102010102010214
:1005D0000102010200020102000200020002010207
:1005E00001010201020102010201020102010201F4
:1005F00002010201020101000102010201020102E5
:1006000001020102010201020100010100000002D9
:1006100002020202000000000202020200000001C9
:1006200001010101010101010101010101010101BA
:1006300001010101010101010101010101010101AA
:10064000010101010101010101010100000001029C
:100650000202020202020202020201000000010183
:100660000001020202000202000000020201020276
:100670000201000101000202020202020202020261
:100680000202020202020200010101020201020151
:100690000202010101020202020102020101010241
:1006A0000202020202020202000002020201020130
:1006B0000201010101020102010202020000020224
:1006C000020202020202020101010202010201020F
:1006D0000201010102020202010202020101000202
:1006E00002020202020202020202020202020202EA
:1006F00000010100010202020102020000000202E8
:1007000001020202010001010000000102020202D6
:1007100002020202020202010000000101010101C5
:1007200001010101010101010101010101010101B9
:1007300001010101010101010101010101010101A9
:100740000101010101010100000002020202020296
:100750000202020202020200000001010002020283
:100760000202000202020202020002020202000170
:10077000010202020202020202020202020202025A
:10078000020202020101020202010202020201014E
:10079000010202020201020202010102020202003F
:1007A0000202020100000202020202020202010130
:1007B000020202020202020200000102020202021E
:1007C000020202010102020201020202020101010F
:1007D00002020202010202020101020202020002FE
:1007E00002020202020200020202020202010100EF
:1007F00002020202020202020202020202020202D9
:1008000002000101000000020202020202020202D2
:1008100002020202000000010101010101010101C7
:1008200001010101010101010101010101010101B8
:1008300001010101010101010101010101010101A8
:100840000101010000000202020202020202020291
:100850000202020000000101000102010201020087
:100860000200020102010201020100010102020272
:100870000202020202020202020202020202020258
:100880000101020102000201020102010200020153
:10089000020102010201010202020202020202023C
:1008A000020201020202020202020101020202002D
:1008B000020202010202020202020002020202011C
:1008C0000102010201020102000201020102010211
:1008D00000020102010102020202020202020202FD
:1008E00002020202020202020201010001020102EE
:1008F00001020102000201020102010201000101E4
:1009000000000002020202020202020202020202CD
:1009100000000001010101010101010101010101CA
:1009200001010101010101010101010101010101B7
:1009300001010101010101010101010101010100A8
:10094000000002020202020202020202020202008D
:10095000000001010002010201000000000001028C
:10096000020202020102000101020202020202026C
:10097000020202020202020002020202010102025B
:10098000010202010202020202020102000102024D
:100990000201010201000000000102020202020243
:1009A000020002020202010102020202000202022D
:1009B0000202020100000000010202010102020124
:1009C000020001020202020202010202010202020C
:1009D00001010202020200020202020202020202FB
:1009E00002020202020101000201020201020201EE
:1009F00000000000000202010200010100000002EC
:100A000002020202020202020202020200000001CD
:100A100001010101010101010101010101010101C6
:100A20000101010101080420C030A04C0A3E0A3136
:100A30000A4A6F696E2028736C6176652900486FD9
:100A4000737420286D6173746572290053696E6731
:100A50006C6520706C61796572000A4E6F2053449A
:100A60002063617264206F720A6E6F204C4F4144A4
:100A700045522E4845580A0A153A45786974001DB2
:100A800020466C617368696E670A20206C6F616430
:100A900065722E2E2E0A0A444F4E2754205455526A
:100AA0004E204F464621000A0A153A49676E6F727A
:100AB00065006D560A0A504C454153452054555225
:100AC0004E204F464620004C4F572042415454453B
:100AD0005259212000172B152010204C4F4144451E
:100AE0005200172B162013140017534400161378C6
:100AF0000016131400151020001520100000540AD1
:100B000003E181867F3E186D830F0F0E018386609F
:100B100033186DC3198F1803C38E6033186DE3301B
:100B2000CF1803C39E603630CDE360CF3006C79E3A
:100B30007E3E30CDB360CF300CC6F6603330D9B6D0
:100B400060CF33CFCCF66061B0DB1E60CF30D86CA5
:100B5000E6C061B0DB1E618F19986CC6C063B19BA3
:100B60000E330F0FB078C6FF7E1F1B061E0F050049
:100B700089300802380249786814000003053F21D3
:100B80003F1208120A100A0E1C0E0C1E0C141A1426
:100B9000161F161E131E1E1B1E1E1F1E3F213F3A30
:100BA0002F3A173D173F213F181F02040A041F0E5A
:100BB00004040E1F0A1F0A0E0E1F04110E2E252EEE
:100BC0002F2A2E262929021F02081F08150E0404A9
:100BD0000E150E15151B151B040604040C0400004D
:100BE000000017000300031F0A1F16371A19041309
:100BF0000A153A000300000E11110E000A040A043F
:100C00000E040030000404040010001804031F1137
:100C10001F121F101D151711151F07041F17151D73
:100C20001F151D01011F1F151F17151F000A0000AA
:100C30003200040A110A0A0A110A040115020E11EF
:100C4000171E051E1F150A0E110A1F110E1F151162
:100C50001F05010E111D1F041F111F1108100F1F6A
:100C6000041B1F10101F061F1E040F0E110E1F095C
:100C7000060E112E1F051A121509011F011F101F44
:100C80000F180F1F0C1F1B041B031C031915130047
:100C90001F11030418111F0002010220202000016F
:100CA000020C121E1F120C0C12120C121F0C1A1422
:100CB000041E05242A1E1F021C141D1020201D1FA7
:100CC0000814111F101E041E1E021C0C120C3E0ADA
:100CD000040C123E1E040214160A020F120E101EFD
:100CE0000E100E1E081E120C1226281E322A260472
:100CF0001E21001F00211E040102013F213FF6E8D2
:100D0000DBCFC3B8AEA49B928A827B746E68625CB0
:100D100057524E4945413E3A3734312E2C2927252A
:100D2000232145006801000005006801380100002A
:100D30000500380168010000400D3C0D0101FF0372
:100D40000101F7030000000800020100000304078E
:100D50000000000000000000010204081020408094
:100D600001020408102001020408102004040404F5
:100D70000404040402020202020203030303030345
:100D800000000000230026002900000000002500CC
:100D900028002B0000000000240027002A00061174
:100DA000092811241FBECFEFD8E0DEBFCDBF12E06F
:100DB000A0E0B1E0E8E9F0E602C005900D92AC34A5
:100DC000B107D9F726E0ACE4B2E001C01D92A2352C
:100DD000B207E1F71DE0C2EADDE004C02297FE01A0
:100DE0000E94D22FCE39D107C9F70E94132E0C943E
:100DF0004A300C9400008DE380934C028091F602FF
:100E0000882311F081E301C080E380934D028EE3DB
:100E100080934E028091F502882311F081E301C096
:100E200080E380934F028FE3809350028091F4021D
:100E3000882311F081E301C080E38093510280E4B4
:100E4000809352028091F302882311F081E301C064
:100E500080E38093530281E4809354028091F202F4
:100E6000882311F081E301C080E38093550282E47E
:100E7000809356028091F102882311F081E301C032
:100E800080E380935702809108028823C9F081E0B3
:100E900080934C0280934D0280934E0280934F02C8
:100EA00080935002809351028093520280935302A8
:100EB0008093540280935502809356028093570288
:100EC0008091EE028823C9F082E080934C028093E7
:100ED0004D0280934E0280934F0280935002809384
:100EE0005102809352028093530280935402809364
:100EF000550280935602809357021092F602109288
:100F0000F5021092F4021092F3021092F202109283
:100F1000F102ECE4F2E0DF010D900020E9F7AD0111
:100F2000415051094C545240E0918505F09186059D
:100F30000280F381E02D6CE472E085E895E009948D
:100F4000DC01ED91FC910190F081E02D09948FEF8F
:100F50008093060284E18093070208950F931F9304
:100F6000CF93DF93162F98E0899FE0011124C55F8E
:100F7000DD4F062F20E04E8160E08CE193E00E947F
:100F8000FA2320E0488161E08CE193E00E94FA239B
:100F90002C8121954D8162E08CE193E00E94FA233F
:100FA0002A812A534B8163E08CE193E00E94FA236B
:100FB000212F4F8169818CE193E0DF91CF911F91C7
:100FC0000F910C942B2420E030E0FA01E20FF31F84
:100FD000948191110DC090E5928390915D0293836D
:100FE00091E094838083618360E081E00C94AE079C
:100FF0002A5F3F4F2432310541F708951F93CF9365
:10100000DF93C0E0D0E014E1FE01EA55FD4F84819A
:10101000882379F08281612F0E94502F963048F00A
:1010200041814E5F60816E5F21E085E493E00E9424
:10103000E71FFE01EE57FD4F8481882379F08281FE
:10104000612F0E94502F963048F041814E5F6081A1
:101050006E5F21E085E493E00E94E71FFE01E25A03
:10106000FD4F8481882379F08281612F0E94502F67
:10107000963048F041814E5F60816E5F21E085E4EB
:1010800093E00E94E71F2696C432D10509F0BCCF39
:10109000DF91CF911F910895E82FF0E085E1689FDF
:1010A000E00DF11D1124E65FFE4F8081813011F0CB
:1010B00092E190839FEF980F81E0923008F080E0FA
:1010C00008951F93CF93DF93EC0160E080E00E94CE
:1010D000AE0782E08093F00283E08093EF0281E02C
:1010E0008D8310E08B81181778F4698167FD6D5F3F
:1010F00065956595888187FD8D5F85958595810FBF
:101100000E944C08882311F010E012C01F5FEACF44
:10111000698167FD6D5F65956595888187FD8D5F48
:1011200085958595811B0E944C08811104C01F5F25
:101130008B81181768F310E010C0698167FD6D5F3F
:1011400065956595610F888187FD8D5F859585958E
:101150000E944C08811104C01F5F8B81181768F32F
:1011600010E010C0698167FD6D5F65956595611B35
:10117000888187FD8D5F859585950E944C0881113A
:1011800004C01F5F8B81181768F3DF91CF911F9107
:1011900008952F923F924F925F926F927F928F921B
:1011A0009F92AF92BF92CF92DF92EF92FF920F93F6
:1011B0001F93CF93DF938AEAE82E82E0F82E96EA17
:1011C000C92E92E0D92E22E6422E22E0522E3EE592
:1011D000232E32E0332EC0E6D2E046E8A42E42E0D1
:1011E000B42E52E8852E52E0952E04E812E068EA0B
:1011F000662E62E0762ED7018C91882309F1F301E7
:101200008081882309F496C03197E081E7FDED5F86
:10121000E595E59585E1E89FF0011124D6018C91D3
:1012200087FD8D5F85958595E65FFE4FE80FF11D83
:101230008081833008F07EC0F301808181508083FB
:10124000D5018C91882309F1F8018081882309F464
:1012500079C03197E081E7FDED5FE595E59585E1A2
:10126000E89FF0011124D4018C9187FD8D5F859555
:101270008595E65FFE4FE80FF11D8081833008F011
:1012800061C0F801808181508083D2018C918823D4
:1012900001F18881882309F45DC0FE013197E08166
:1012A000E7FDED5FE595E595B5E1EB9FF0011124D4
:1012B000D1018C9187FD8D5F85958595E65FFE4F09
:1012C000E80FF11D8081833008F044C0888181508F
:1012D0008883B6E0EB0EF11CE6E0CE0ED11CF6E002
:1012E0004F0E511C86E0280E311C2696A6E0AA0E51
:1012F000B11CB6E08B0E911C0A5F1F4FE6E06E0E2C
:10130000711CFEECEF16F2E0FF0609F074CFDF91DE
:10131000CF911F910F91FF90EF90DF90CF90BF90F2
:10132000AF909F908F907F906F905F904F903F9085
:101330002F900895D3011C92F7011082C6010E94DC
:1013400061087ACFD8011C92F5011082C4010E9475
:10135000610897CF1882D2011C92C1010E946108D6
:10136000B5CF0F931F93CF938091EF02882309F499
:101370006AC081508093EF028091F00290E09C015E
:101380002F5F3F4F442737FD4095542F662777271F
:10139000681B790B882777FD8095982F0E94AF2DC9
:1013A00020915A0230915B028901222717FD209576
:1013B000322F060F171F281F391F10935B0200934F
:1013C0005A028091F00290E09C012F5F3F4F44272A
:1013D00037FD4095542F66277727681B790B8827A0
:1013E00077FD8095982F0E94AF2D20915802309163
:1013F00059028901222717FD2095322F060F171F4A
:10140000281F391F10935902009358028091FC0243
:1014100086958695C091FA022091F002829F9001F4
:101420001124442737FD4095542F60E070E0CB0134
:101430000E94AF2DC61B6C2F87EF92E0CF911F91BA
:101440000F910C94711C10925B0210925A02109230
:10145000590210925802CF911F910F9108958F92C7
:101460009F92BF92CF92DF92EF92FF920F931F93C2
:10147000CF93DF931F92CDB7DEB70E94B1097AE018
:10148000E72E71E0F72EC12CBB24B394BC0CD12CF9
:10149000812C912C8701080D191DF80150815523CD
:1014A00069F1513079F4809158024C2D481B80919C
:1014B0005A026D2D681B04E024E085E493E00E944D
:1014C000D81E1CC05B3088F025E23AE04C2D6D2D13
:1014D00085E493E059830E94A020598151505A30ED
:1014E00009F450E0F801508309C002E022E04B2DDE
:1014F00061E06D0D85E493E00E94B01EFFEF8F1A4E
:101500009F0A84E0D80EE4E5DE12C4CFF5E1EF0EC9
:10151000F11CC80E80E3C812B7CF0F90DF91CF91B6
:101520001F910F91FF90EF90DF90CF90BF909F9011
:101530008F900895CF93DF9320E030E040E050E0BB
:10154000DC01A20FB31FB901665F7E4FFA01EA0FFB
:10155000FB1FE491EB01C40FD51FE8834F5F5F4F82
:101560004531510599F72B5E3F4F2C3F310531F73F
:10157000DF91CF910895823089F02CF4882341F0D7
:10158000813049F00895833061F0843069F0089526
:1015900089E299E00BC08DE298E008C081E397E012
:1015A00005C085E396E002C089E395E00C949A0AB1
:1015B000482F20E030E0F901EA55FD4F848188236F
:1015C00071F0908197FD9D5F95959595941307C057
:1015D000918197FD9D5F95959595961779F1F90104
:1015E000EE57FD4F8481882371F0908197FD9D5FB8
:1015F00095959595941307C0918197FD9D5F95955D
:1016000095959617D9F0F901E25AFD4F8481882308
:1016100071F0908197FD9D5F95959595941307C006
:10162000918197FD9D5F95959595961739F02A5F65
:101630003F4F2432310509F0BECF80E0089584E0A9
:101640008093E4028093E50281E08093E602809338
:10165000E7028093E9021092EA0208958CE48093F5
:10166000DD0288E28093DE0283E18093DF028AE07C
:101670008093E00281E08093E2021092E3020895F9
:1016800084E08093D60288E28093D70281E0809341
:10169000D8029AE09093D9028093DB028093DC0217
:1016A00008958CE48093CF0284E08093D00283E19C
:1016B0008093D10281E08093D2028093D402809300
:1016C000D502089510925C020E941F0B0E942E0BFF
:1016D0000E94400B0E94510B83E080935D0280E0EA
:1016E00090E0FC01EA55FD4F1482FC01EE57FD4FDE
:1016F0001482FC01E25AFD4F148206968432910551
:1017000081F708950F93CF93DF93CDB7DEB7279777
:101710000FB6F894DEBF0FBECDBF8F83622F432F6D
:101720007723C9F0811108C0002319F022E335E0C6
:1017300005C02BE235E002C024E235E085E493E009
:1017400027960FB6F894DEBF0FBECDBFDF91CF91C5
:101750000F910C94A02027960FB6F894DEBF0FBE11
:10176000CDBFDF91CF910F9108950F9301E02091AC
:10177000E4023091E5024091E6025091E702609167
:10178000E8027091E9028091EA020E94820B809146
:10179000EB02811111C000E02091DD023091DE02E8
:1017A0004091DF025091E0026091E1027091E2020B
:1017B0008091E3020E94820B00E02091D6023091DA
:1017C000D7024091D8025091D9026091DA0270910B
:1017D000DB028091DC020E94820B2091CF023091CB
:1017E000D0024091D1025091D2026091D302709107
:1017F000D4028091D5020E94820B0F910895CF935D
:10180000C42F0E94D80A2AE030E040E050E088234C
:1018100061F060E070E0CB010E94AF2D25E330E085
:101820002C1B3109260F371F06C060E070E0CB018A
:101830000E94AF2D9B01C901CF910895DF92EF92D5
:10184000FF920F931F93CF93DF93F82EE62E85E13F
:10185000689F80011124D12CC0E0D0E0065F1E4FAC
:101860008D2D8F0DF801E80FF11D90819150923070
:1018700010F4D12C15C04D2D6E2D0E94FF0BC80FFA
:10188000D91FD39483E0D812EBCFF3CF4D2D6E2D1B
:101890000E94FF0BC80FD91FD39483E0D81649F0DC
:1018A0008F2D8D19F801E80FF11D90819150923024
:1018B00068F7D12C0F2D10E0065F1E4F0AC04D2D8A
:1018C0008F2D0E94FF0BC80FD91FD39483E0D81629
:1018D00061F06D2D6E0DF80185E1689FE00DF11D41
:1018E000112480818150823050F7D12C0AC04D2DB7
:1018F0008F2D0E94FF0BC80FD91FD39483E0D816F9
:1019000061F06E2D6D19F80185E1689FE00DF11D04
:10191000112480818150823050F7CE01DF91CF9128
:101920001F910F91FF90EF90DF9008950F931F93F9
:10193000CF93DF93EC018B018FE097E2998388834B
:101940009B838A839D838C839F838E83FB0163812A
:101950006F5F828195E1699FF0011124E65FFE4F80
:10196000E80FF11D9081911104C00E941E0C998313
:101970008883F801638182818F5F95E1699FF0011F
:101980001124E65FFE4FE80FF11D9081911104C014
:101990000E941E0C9B838A83F801638161508281BF
:1019A00095E1699FF0011124E65FFE4FE80FF11DFC
:1019B0009081911104C00E941E0C9D838C83F801BC
:1019C00063818281815095E1699FF0011124E65F76
:1019D000FE4FE80FF11D9081911104C00E941E0C72
:1019E0009F838E83DF91CF911F910F910895CF92A6
:1019F000DF92EF92FF920F931F93CF93DF93CDB7B8
:101A0000DEB727970FB6F894DEBF0FBECDBF142FF9
:101A1000F52E16160CF461C0652F842F0E94D80A8B
:101A200081115BC0CC24CA94C10E6F2D8C2D0E94F5
:101A30001E0CC3970CF051C0DD24D394D10E6F2D32
:101A40008D2D0E941E0CC3970CF047C0EE24EA9423
:101A5000EF0C6E2D812F0E941E0CC397F4F501E050
:101A60000F0D602F812F0E941E0CC397B4F52EE13D
:101A700030E040E050E060E070E0CB010E94AF2D2C
:101A8000672B682B692B59F185E1F89E9001112491
:101A9000265F3E4FF901EC0DF11D80818230F9F097
:101AA000F901ED0DF11D80818230C9F0412F50E028
:101AB000465F5E4FFA0185E1E89EE00DF11D1124BD
:101AC0008081823061F0FA0185E1089FE00DF11D0F
:101AD000112481E09081923019F080E001C081E012
:101AE00027960FB6F894DEBF0FBECDBFDF91CF9122
:101AF0001F910F91FF90EF90DF90CF900895EF929C
:101B0000FF920F931F93CF93DF93CDB7DEB7289744
:101B10000FB6F894DEBF0FBECDBF8C0180910802D6
:101B20008111CBC0D80115968C911597882309F4A3
:101B3000C4C012968C9112972C91332727FD3095B3
:101B4000B4E08B02C00111242817390709F0B5C091
:101B5000F80183812181332727FD3095F4E08F023E
:101B6000C00111242817390709F0A7C0B801CE0118
:101B700001960E94960CFE01319620E030E076E955
:101B800060E04FE057E279018191919184179507C8
:101B90001CF0CA01E72EF62E2F5F3F4F243031058F
:101BA00021F07E2D6F2DAC01EECFC3975CF0D801F4
:101BB00013966C91139712968C910E941E0CC297EB
:101BC0000CF47BC0F1E0EF16F10409F04DC0D80130
:101BD0001396EC91139712968C918F5F0BC093E044
:101BE000E916F104A1F4D8011396EC91139712961B
:101BF0008C918150B5E1EB9FF0011124E65FFE4F1F
:101C0000E80FF11D9081911102C0F8018283D80183
:101C10002C9111963C91119712964C911297139614
:101C20005C91139714966C91149715967C91159767
:101C300016968C910E94F70CF801882379F0638145
:101C4000660F660F82814EE552E0880F880F0E9472
:101C5000E30782E1D80114968C932FC08481181673
:101C600064F58150848329C042E0E416F10454F401
:101C7000EF2869F6F80183818F5F45E1849FF001C9
:101C800011240DC082E0E816F10409F0A8CFD801B4
:101C900013968C918150B5E18B9FF0011124D801EE
:101CA00012969C911297E65FFE4FE90FF11D90810D
:101CB0009111ADCF13968C93AACF28960FB6F894B6
:101CC000DEBF0FBECDBFDF91CF911F910F91FF906F
:101CD000EF90089586ED92E00E947F0D8FEC92E0E8
:101CE0000C947F0DFC0185818823B1F14081842F04
:101CF000992787FD9095528164E056029001112446
:101D0000A3818217930769F44181842F992787FD66
:101D1000909564E0A602900111248217930749F47C
:101D20000FC08217930714F44F5F01C041504083E6
:101D300007C08217930714F44F5F01C041504183DD
:101D400085E1A89FD0011124A65FBE4FA50FB11D4C
:101D50008C918B3008F015820895FC0185818823D1
:101D6000E9F180910802811139C041E062E081E02F
:101D700093E00E94761D882321F081E08093F30296
:101D800023C041E060E081E093E00E94761D88235B
:101D900021F081E08093F40217C041E061E081E02E
:101DA00093E00E94761D882321F081E08093F60263
:101DB0000BC041E063E081E093E00E94761D882340
:101DC00019F081E08093F50264E081E093E00E94E5
:101DD0005F1D882319F081E08093F2020895CF936C
:101DE000DF93FC01D381C2816D2F8C2F0E94D80A12
:101DF000811113C09091EE026D2F660F660F8C2F2C
:101E0000880F880F992319F046EA52E002C042E891
:101E100052E0DF91CF910C94E307DF91CF910895C9
:101E2000CF93DF93C82FD62F0E94D80A81110DC0FF
:101E300085E1D89FF0011124E65FFE4FEC0FF11D04
:101E40009081915081E09A3008F480E0DF91CF9149
:101E500008951F93CF93DF93EC018A814881552722
:101E600047FD509594E089029001112442175307D1
:101E700091F41B814981552747FD509594E0190243
:101E8000900111244217530731F41150612F0E9421
:101E9000100F81111B83DF91CF911F9108951F9324
:101EA000CF93DF93EC018A814881552747FD5095F8
:101EB00094E08902900111244217530791F41B8189
:101EC0004981552747FD509594E01902900111244E
:101ED0004217530731F41F5F612F0E94100F8111C9
:101EE0001B83DF91CF911F9108951F93CF93DF93B1
:101EF000EC011A814881552747FD509584E018026E
:101F0000900111244217530791F46B8149815527A1
:101F100047FD509584E06802900111244217530751
:101F200031F41150812F0E94100F81111A83DF911B
:101F3000CF911F9108951F93CF93DF93EC011A81E6
:101F40004881552747FD509584E0180290011124DF
:101F50004217530791F46B814981552747FD5095EE
:101F600084E06802900111244217530731F41F5F87
:101F7000812F0E94100F81111A83DF91CF911F9141
:101F80000895CF93DF93EC018D81882309F43FC03E
:101F90008091080281113BC041E062E081E093E062
:101FA0000E94761D882321F0CE010E949B0F23C042
:101FB00041E060E081E093E00E94761D882321F0FB
:101FC000CE010E94750F17C041E061E081E093E00F
:101FD0000E94761D882321F0CE010E94290F0BC09C
:101FE00041E063E081E093E00E94761D882319F0D0
:101FF000CE010E944F0F64E081E093E00E945F1DDC
:10200000882329F0CE01DF91CF910C94EF0EDF9160
:10201000CF91089529EF33E040E060E085E493E05C
:102020000E94A0208AE080934E038AE280934F03AF
:1020300060EB70E085E493E00E94972C64E081E01F
:1020400093E00E945F1D81110EC065E081E093E086
:102050000E945F1D811107C066E081E093E00E944D
:102060005F1D882319F083E38093070208951F936F
:10207000CF93DF9327EE31E040E060E085E493E02A
:102080000E94A020CAECD2E016E14991442359F005
:10209000440F440F440F4A5F20EE31E0612F85E486
:1020A00093E00E94A0201A5F143379F764E081E086
:1020B00093E00E945F1D811107C065E081E093E01D
:1020C0000E945F1D882339F080910602853074F4E8
:1020D00081E08093070266E081E093E00E945F1D4B
:1020E000882331F082E38093070202C082E3F1CFBC
:1020F000DF91CF911F9108950F930E942F0A0E94A4
:10210000B50B0E94FE0760E085E493E00E94621E2A
:1021100020915C02220F00E340E060E085E493E060
:102120000E94D81E80915C02282F220F6AE270E084
:10213000681B710987FD7395660F40E085E493E0A5
:102140000E94D81E40E061E085E493E00E94661E94
:102150008CE080934E0381E080934F0380915C027A
:102160008F5F80935C028F3119F48BE080930702BC
:102170000F91089585E895E00C945A2762E070E08D
:1021800085E895E00E94772762EA71E185E895E0AD
:102190000E94FF276BEF76E085E895E00C94042819
:1021A000CF9310920802C4E18091EC02811114C017
:1021B00061E070E080E090E00E94A72AC150A1F7A2
:1021C00042E069E770E087EF92E00E94761681E0D6
:1021D0008093ED02809308021092EC02CF91089553
:1021E0006EEB70E087EF92E00E94821B0E94A707CF
:1021F0000C94620B87EF92E00E94FE1B0E94F0108D
:1022000010920F030E94BA100C94BE101092480353
:102210001092470386E292E0909346038093450331
:102220000895CF93DF934CE050E062E070E085E8E2
:1022300095E00E94F927882309F475C01092ED02F9
:1022400010920802D1E085E895E00E949426892B3F
:1022500009F475C085E895E00E949C26C82F8E334E
:1022600049F18CF4823009F454C08D33C1F08130CF
:1022700051F742E063EA70E087EF92E00E94761641
:10228000C0930802E0CF803461F1FCF08134A9F101
:102290008234C9F685E895E00E949C26D4CF85E873
:1022A00095E00E949C26C19771F68DED92E00E9408
:1022B000290FC9CF85E895E00E949C26C19719F6A1
:1022C0008DED92E00E944F0FBECF85E895E00E9411
:1022D0009C26C19709F0B7CF8DED92E00E94750F53
:1022E000B2CF85E895E00E949C26C19709F0ABCF5C
:1022F0008DED92E00E949B0FA6CF85E895E00E94AD
:102300009C26C19709F09FCF8DED92E00E94EF0EC1
:102310009ACF42E066E970E087EF92E00E9476167D
:10232000D093080290CF42E063E870E087EF92E03C
:102330000E94761681E0809308028093ED02DF917F
:10234000CF910895AF92BF92CF92DF92EF92FF921A
:102350000F931F93CF93DF93BB24B394E0E5AE2E8E
:10236000F6E0FF2E85E895E00E949426892B09F47B
:1023700026C185E895E00E949C26803209F48DC034
:102380004CF5843109F469C0A4F48A3009F44CC0D6
:102390004CF4833039F785E895E00E949C268093C1
:1023A0000702E0CF8B3009F446C08C3009F44AC0F4
:1023B000D9CF863109F45FC00CF456C08E3109F4D0
:1023C00065C08F3179F685E895E00E949C26809360
:1023D000D702C8CF863409F497C0ACF4893209F427
:1023E00067C054F4883209F0BDCF85E895E00E94BB
:1023F0009C268093CF02B6CF8A3209F460C0823324
:1024000009F468C0AFCF883409F478C00CF4A5C0D3
:10241000893409F4CEC08A3409F0A4CF85E895E068
:102420000E949C26E82E9ECF85E895E00E949C267F
:102430008093E40297CF85E895E00E949C268093E4
:10244000E50290CF85E895E00E949C2621E0C197A7
:1024500009F020E02093E90285CF85E895E00E940D
:102460009C268093DD027ECF85E895E00E949C2625
:102470008093DE0277CF85E895E00E949C2621E0DC
:10248000C19709F020E02093E2026CCF85E895E047
:102490000E949C268093D60265CF85E895E00E9435
:1024A0009C2621E0C19709F020E02093DB025ACF5F
:1024B00085E895E00E949C268093D00253CF85E862
:1024C00095E00E949C2621E0C19709F020E020932E
:1024D000D40248CF85E895E00E949C2660910602D0
:1024E000772767FD7095AC0155276417750709F4C8
:1024F00039CF809306020E94BB0A34CF85E895E06D
:102500000E949C26D82E2ECF45E06DE670E087EF26
:1025100092E00E94761685E895E00E949C268A301B
:1025200030F48F9DE0011124CA55DD4F11C0843174
:1025300038F48A50F89EE0011124CE57DD4F08C0D0
:102540008E3130F48451F89EE0011124C25ADD4FDF
:10255000AA82BC82C882E98205CF45E068E670E0C5
:1025600087EF92E00E94761685E895E00E949C260F
:10257000982F8A3030F49F9D800111240A551D4FF9
:1025800011C0843138F49A50F99E800111240E57FD
:102590001D4F08C08E3130F49451F99E80011124F2
:1025A000025A1D4FF8011482D382C8010E946108AB
:1025B000D9CE85E895E00E949C26C82ED3CE81E036
:1025C0008093EC021092ED02DF91CF911F910F9159
:1025D000FF90EF90DF90CF90BF90AF9008956F92F3
:1025E0007F928F929F92AF92BF92CF92DF92EF92A3
:1025F000FF920F931F93CF93DF9362E070E085E823
:1026000095E00E94832703E612E0B8EAEB2EB2E0E1
:10261000FB2EC7E8D2E08BEAA82E82E0B82E9AE023
:10262000892E912C24E1C22ED12C34E1732EACEEF4
:102630006A2E6C0CF50131978081882399F1F7019E
:102640008081672D0E94502F963060F169E470E020
:1026500085E895E00E94A007F7013297608177270F
:1026600067FD709585E895E00E94A0076AE470E038
:1026700085E895E00E94A007F70131978081682FD7
:10268000772767FD709585E895E00E94A00766E4CE
:1026900070E085E895E00E94A007662D85E895E04A
:1026A0000E941B27F50180818823C9F0108268E40D
:1026B00070E085E895E00E94A007F50132976081FF
:1026C00085E895E00E941B2767E470E085E895E0C7
:1026D0000E94A007662D85E895E00E941B27FE0159
:1026E00031978081882391F1F7018081672D0E94C5
:1026F000502F963058F169E470E085E895E00E942B
:10270000A007FE0135976081772767FD709585E802
:1027100095E00E94A0076AE470E085E895E00E94D9
:10272000A007FE0134976081772767FD709585E8E3
:1027300095E00E94A00766E470E085E895E00E94BD
:10274000A007B40185E895E00E94A007888188234E
:10275000C9F0188268E470E085E895E00E94A0075F
:10276000FE013297608185E895E00E941B2767E4AF
:1027700070E085E895E00E94A007B40185E895E047
:102780000E94A007F80131978081882399F1F70111
:102790008081672D0E94502F963060F169E470E0CF
:1027A00085E895E00E94A007F801359760817727BA
:1027B00067FD709585E895E00E94A0076AE470E0E7
:1027C00085E895E00E94A007F80134978081682F82
:1027D000772767FD709585E895E00E94A00766E47D
:1027E00070E085E895E00E94A007B60185E895E0D5
:1027F0000E94A007F80180818823C9F0108268E454
:1028000070E085E895E00E94A007F80132976081AA
:1028100085E895E00E941B2767E470E085E895E075
:102820000E94A007B60185E895E00E94A0070A5F14
:102830001F4FFFEFCF1ADF0A86E0E80EF11C269645
:10284000EFEF8E1A9E0AF6E0AF0EB11C8AE1C816B1
:10285000D10409F0ECCE63E070E085E895E00E94D9
:10286000A0076091070285E895E00E941B2762E3BC
:1028700070E085E895E00E94A00760910602772746
:1028800067FD709585E895E00E94A0076AE070E01A
:1028900085E895E00E94A0076091E402772767FD34
:1028A000709585E895E00E94A0076BE070E085E8F0
:1028B00095E00E94A0076091E502772767FD70957B
:1028C00085E895E00E94A0076CE070E085E895E05F
:1028D0000E94A0078091E902882319F061E370E06B
:1028E00002C060E370E085E895E00E94A00764E123
:1028F00070E085E895E00E94A0076091DD027727EF
:1029000067FD709585E895E00E94A00765E170E09D
:1029100085E895E00E94A0076091DE02772767FDB9
:10292000709585E895E00E94A00766E170E085E873
:1029300095E00E94A0078091E202882319F061E3EC
:1029400070E002C060E370E085E895E00E94A007B7
:102950006EE170E085E895E00E94A0076091D602E4
:10296000772767FD709585E895E00E94A0076FE1E5
:1029700070E085E895E00E94A0076091D702772774
:1029800067FD709585E895E00E94A00760E270E021
:1029900085E895E00E94A0078091DB02882319F06A
:1029A00061E370E002C060E370E085E895E00E94BA
:1029B000A00768E270E085E895E00E94A0076091BA
:1029C000CF02772767FD709585E895E00E94A00704
:1029D00069E270E085E895E00E94A0076091D0026E
:1029E000772767FD709585E895E00E94A0076AE269
:1029F00070E085E895E00E94A0078091D4028823CA
:102A000019F061E370E002C060E370E085E895E0F2
:102A10000E94A00785E895E0DF91CF911F910F916B
:102A2000FF90EF90DF90CF90BF90AF909F908F90EE
:102A30007F906F900C94FC270E9411110C94EF1260
:102A40008091EB02811107C08091EE0281110C94FC
:102A50001C150C94D0100895CF93DF9387EF92E06C
:102A60000E943017882309F408C18091070284313D
:102A700069F5C1E0C093080243E06BE27AE087EFBA
:102A800092E00E943D18813079F08230B1F08111DE
:102A9000F0C010920802C093ED02C093EE02C09302
:102AA000EB02C0930702E9C0109208021092ED02F7
:102AB0008093EE021092EB02A6C0109208021092D0
:102AC000ED021092EE021092EB02D7C081119EC06F
:102AD00066E081E093E00E945F1D882319F083E3A4
:102AE000809307028091EE028823F9F084EE92E051
:102AF0000E94C10F0E946A0E8091EB02811106C0F4
:102B00000E941C158DED92E00E94720E84EE92E000
:102B10000E94720E86ED92E00E94720E8FEC92E09F
:102B20000E94720E0E94C9080AC08091EB028111B6
:102B300006C08DED92E00E94AD0E0E94D0100E9462
:102B40002F0A0E94B50B0E94FE078091E90288239C
:102B5000D1F08091E202882369F08091EB02882312
:102B600009F48BC08091DB02811187C08091D4026F
:102B7000811183C0E0910602FF27E7FDF095E6533F
:102B8000FD4F81E03EC08091EB0281110DC080912C
:102B9000E202882349F0E0910602FF27E7FDF09565
:102BA000E653FD4F82E02DC09091DB028091D4026C
:102BB0009923E9F0E0910602882391F0CE2FDD27DA
:102BC000C7FDD09525E030E040E050E063E070E0E4
:102BD00080E090E00E94AF2DC653DD4F688312C0A5
:102BE000FF27E7FDF095E653FD4F83E00AC08823F9
:102BF00049F0E0910602FF27E7FDF095E653FD4F0F
:102C000084E080838AE08093070237C08B3031F400
:102C10000E942015DF91CF910C9437108A3031F447
:102C20000E942015DF91CF910C947C108C30C1F361
:102C3000813099F40E9420158091EE028823E9F0FA
:102C40000E94620B10920702809106028F5F8093B0
:102C50000602DF91CF910C94BB0A823331F40E94BB
:102C60002015DF91CF910C940A10833331F40E9428
:102C70002015DF91CF910C94F010DF91CF91089542
:102C8000CF93CFB7F89480917E03811127C0E6E7F8
:102C9000FDE08491E2E6FDE09491E82FF0E0EE0F94
:102CA000FF1FEC56F24FA591B4918C91892321F42A
:102CB00061E08AE00E94FA2B61E08AE00E94C12B69
:102CC0008CB580618CBD8CB580648CBD61E08DE07D
:102CD0000E94C12B61E08BE00E94C12B80917E039A
:102CE0008F5F80937E03CFBFCF910895FC01EC5797
:102CF000FF4F718360833296445F408308958F92C3
:102D00009F92AF92BF92CF92DF92EF92FF920F937A
:102D10001F93CF93DF93EC015C0186E8A80EB11CF2
:102D2000D5018C91882309F44DC08C3018F41CE037
:102D3000181B01C010E0FE01EA5AFF4F81E08083BA
:102D40006E01BEE4CB0ED11C60E0C6010E94621E83
:102D50004E01E3E58E0E911CD4018C9103E0080F27
:102D60009DE2F92E4F2D481B410F23E0E22E24E572
:102D700060E0C6010E94672061E0C6010E94621EF9
:102D8000F401808103E0080F4F2D481B410F24E51B
:102D900060E0C6010E940720FE01E95AFF4F84E06F
:102DA00080833196D4018C91181B115D1083CC5710
:102DB000DF4F68817981C6010E94972CF5018081DF
:102DC00081508083DF91CF911F910F91FF90EF9001
:102DD000DF90CF90BF90AF909F908F9008950F930A
:102DE0001F93CF93DF938C01EC01C25BDF4FCE01C9
:102DF0000E94091E6FE77AE0CE010E94972CCE0157
:102E00000E941A1E8CB583608CBD8DB58E7F8DBDE2
:102E10008BE192E0EEEFFFE30995F801EC5AFF4FEA
:102E200010826AE57AE0CE010E94C52CCE010E9494
:102E30001A1E065F1F4FC8010E94281D64E0C801CA
:102E40000E945F1D811107C062E370E080E090E0A6
:102E50000E94A72AF0CFDF91CF911F910F91089583
:102E60008F929F92AF92BF92EF92FF920F931F9318
:102E7000CF93DF93EC017C0100E8E00EF11CF70139
:102E800080809180A280B3800E94782A950184017D
:102E9000061B170B280B390BB901A8015E011FE7B0
:102EA000A10EB11CF501808190E0A0E0B0E08E01A0
:102EB00005581F4F84179507A607B70750F4F80168
:102EC00080819181A281B381892B8A2B8B2B09F080
:102ED0006DC0F80180819181A281B381892B8A2BF9
:102EE0008B2B09F061C05E01FAE0AF0EB11C41E02E
:102EF00066E0C5010E94761D9E012B5D3F4F790162
:102F0000882331F065E0C5010E945F1D811185C0F5
:102F100041E066E0C5010E94761D882331F064E03F
:102F2000C5010E945F1D81118EC041E066E0C501B0
:102F30000E94761D882339F048E264E0C5010E94B2
:102F4000681D81118BC0C7010E94AF24C7010E9478
:102F50001C25C7010E94EC25CE010E947F16CE01E0
:102F60000E948F197E013EE4E30EF11CC7010E940E
:102F70001A1EFE01EC5AFF4F8081811103C0C70168
:102F80000E94091E0E94842AF80160837183828353
:102F90009383FE01EB58FF4FC958DF4F28813981D9
:102FA000621B730B7183608380E05CC00E94782A8F
:102FB000F5012081620F711D811D911DF701608354
:102FC000718382839383FE01EF58FF4F40815181CB
:102FD000628173814F5F5F4F6F4F7F4F408351839B
:102FE00062837383F80110821182128213820E941D
:102FF000842AFE01E958FF4F6083718382839383A3
:10300000CE010E94751CCE010A960E94281DCE0199
:1030100048960E94DE1C81E025C0C7010E949126CF
:1030200061E0680FC7010E947E2682EE9AE0FE01F1
:10303000EC57FF4F9183808388E432968083C701E9
:103040000E94682665CF85ED9AE0FE01EC57FF4FA0
:103050009183808388E43296808367CFCE010E947B
:10306000EF1671CFDF91CF911F910F91FF90EF90ED
:10307000BF90AF909F908F9008952F923F924F9264
:103080005F926F927F928F929F92AF92BF92CF92F8
:10309000DF92EF92FF920F931F93CF93DF93CDB701
:1030A000DEB766970FB6F894DEBF0FBECDBF9E8B1E
:1030B0008D8B6F87788B942EFC01EC5AFF4F10821A
:1030C00088248A941C82A12C30E33B83B12C6C01B0
:1030D0008AE0C80ED11C6D887E8893E5690E711C4C
:1030E000ED89FE89B5962F01242F30E03A87298794
:1030F0008D899E89895A9F4F9E838D83ED89FE8994
:10310000E85AFF4FF887EF832D893E892A5A3F4FAF
:103110003C872B878D899E898B5A9F4F9E878D87F1
:10312000ED89FE89E25BFF4F1F018D899E890E9418
:1031300030178823D1F364E0C6010E945F1D3B81F4
:10314000032F112707FD109581113EC065E0C601D0
:103150000E945F1D811138C066E0C6010E945F1D9C
:10316000811132C03C81311142C044E063E0C601AC
:103170000E94761D882321F0B394C2010E94682624
:1031800044E061E0C6010E94761D882321F0BA94D4
:10319000C2010E9468268B2D992787FD9095E985AD
:1031A000FA858E179F0731F0B7FE05C0BB24BA948D
:1031B000B90C01C0B12CF301808154E0A52EA80EFA
:1031C0008B9DA01811241DC0F301A08064E0C601EE
:1031D0000E945F1D882309F484C0C2010E943C261E
:1031E0008B2CA194A99CA02C1124AA94AA94C80168
:1031F0008A199109A7FC939502970CF476C031E0E7
:103200003C830A0D111DA7FC1A9517FF02C00F5F22
:103210001F4FC801959587959A83898329812B83B0
:10322000ED81FE811082EF81F885808381E0EB855E
:10323000FC858083ED85FE8510820F851889E12C41
:10324000F12C4B2D552747FD509533E0E91420F51F
:10325000E416F50669F4ED81FE813083F301808187
:10326000F22FB89EF00D11248F2FEF81F885808307
:10327000F80165917491C101298B3C8B4A8B5B8B62
:103280000E94C52CFFEFEF1AFF0A0E5F1F4F5B89EC
:103290004A893C892989DACF60E0C1010E94621E17
:1032A000F30180814981B89E400D1124415024E5ED
:1032B00060E0C1010E948D1E61E0C1010E94621E9A
:1032C000F301808103E0080F4981B89E400D11246D
:1032D000425033E0E32E24E560E0C1010E94072064
:1032E00024CFC2010E9452267CCF882D66960FB64D
:1032F000F894DEBF0FBECDBFDF91CF911F910F912C
:10330000FF90EF90DF90CF90BF90AF909F908F9005
:103310007F906F905F904F903F902F900895DF9235
:10332000EF92FF920F931F93CF93DF93EC018C8D5D
:103330009D8D892B09F49CC08E01025B1F4F40E0DC
:1033400061E0C8010E94661E85E5FE01EE5AFF4F4E
:103350009081891B3596808331961082698D61300A
:1033600009F462C028F0888D653008F074C06FC021
:10337000CE0185960E94B22481E0FE01EA5AFF4FF9
:1033800080836CE77BE0C8010E94D2211D8E1C8ED9
:10339000FE01EC5AFF4F108288EAD82E7E018AE0A7
:1033A000E80EF11CCE010E9430178823D9F367EC98
:1033B0007AE0C8010E94972C6A8D7B8D4AE050E02C
:1033C000C8010E94852D62EB7AE0C8010E94972C0B
:1033D0006D2D62956F7070E04AE050E0C8010E9468
:1033E000702D67EA7AE0C8010E94972C64E0C7015B
:1033F0000E945F1D81113CC0DA94A1F660E0CE010D
:103400000E94711C83B7817F846083BF83B7816012
:1034100083BF83B7816083BF889583B78E7F83BF67
:1034200083B78E7F83BFBECFCF58DF4F488159818E
:103430006A817B814F705527662777274830510571
:103440006105710510F467E009C068E707C08823CB
:1034500079F06B5F03C0882359F06FE2C801DF91F8
:10346000CF911F910F91FF90EF90DF900C94BA2CA9
:10347000DF91CF911F910F91FF90EF90DF90089512
:103480002F923F924F925F926F927F928F929F9274
:10349000AF92BF92CF92DF92EF92FF920F931F9362
:1034A000CF93DF93CDB7DEB729970FB6F894DEBF81
:1034B0000FBECDBF998788877C836B831A012C014F
:1034C00080E7480E511CF2018081882309F401C174
:1034D00081E0E885F985EA5AFF4F8083E885F98520
:1034E000EB5AFF4F1082E885F985EC5AFF4F1082A6
:1034F000E885F985108E8F01025B1F4F61E0C801DE
:103500000E94621E888599858D5A9F4F9A83898370
:10351000C884D98497E5C90ED11CE884F984E8E50C
:10352000EE0EF11C68847984F2E56F0E711C8885BB
:1035300099858F589F4F9E838D83A884B9849AE084
:10354000A90EB11C88849984E5E28E0E911C8885B1
:1035500099850E9430178823D1F3EB81FC818491F7
:10356000882321F0E981FA81508101C050E02EEFDB
:103570003AE040E060E0C8015F830E94A0205F81E4
:103580002114310439F04CE0450F910160E0C8018D
:103590000E94A020F60110828CE0F70180836B81ED
:1035A0007C81C8010E94972CF3019081892F880F9C
:1035B000890F81958D5AF6018083E981FA81908186
:1035C000892F880F890F8195835DF7018083ED81B5
:1035D000FE81808184FF03C069EF7AE002C065EF5D
:1035E0007AE0C8010E94C52CF3019081892F880FD1
:1035F000890F81958D5AF6018083F70180818F5F55
:103600008083E885F98582A5882319F061EF7AE047
:1036100002C06DEE7AE0C8010E94C52CF3019081D2
:10362000892F880F890F81958D5AF6018083F701C4
:1036300080818F5F808369EE7AE0C8010E94C52C8B
:1036400065E0C5010E945F1D882359F0C4010E94F6
:10365000912661E0680FC4010E947E26C4010E9489
:10366000682664E0C5010E945F1D811113C0F2014C
:103670002081822F90E0A0E0B0E0ED81FE814081CA
:10368000518162817381481759076A077B07A8F047
:103690002F3F99F08FEFF2018083088519850B5D2C
:1036A0001F4F60E0C8010E945924C8010E943C26B7
:1036B00081E0E885F985808F0CC066E0C5010E9435
:1036C0005F1D882309F443CF888599850E94EF16F2
:1036D00034CF29960FB6F894DEBF0FBECDBFDF9171
:1036E000CF911F910F91FF90EF90DF90CF90BF90FF
:1036F000AF909F908F907F906F905F904F903F9092
:103700002F900895AB016DEF7AE00C94401AE0E839
:10371000F7E72591349181E02130304C09F080E0C9
:103720000895CF93DF93EC010E94871B9E01275AD7
:103730003F4FDE01A059BF4F882309F43AC0E6E9A4
:10374000F7E78491F9018083E7E9F7E7E491EC83F7
:10375000E8E9F7E7E491ED83E9E9F7E785919491EA
:103760009F838E83EBE9F7E785919491998788870A
:1037700087E08BA7EEE9F7E7E491EAA7EFE9F7E73F
:10378000E491EC93E0EAF7E7859194919D8F8C8F1B
:10379000E2EAF7E7859194919F8F8E8FE4EAF7E74D
:1037A0008591949199A388A3E6EAF7E7859194918E
:1037B00020C08CE3F90180831C822FEF2D8380E2EF
:1037C00093E09F838E8384ED93E09987888787E0D9
:1037D0008BA78AA72C938CEA9DE09D8F8C8F8EED12
:1037E0009DE09F8F8E8F84E79EE099A388A38CE352
:1037F0009FE09BA38AA3DF91CF910895AF92BF92E0
:10380000CF92DF92EF920F931F93CF93DF93EC0150
:10381000FC01E158FF4F82E38083349741E050E0A0
:1038200060E070E040835183628373833B978FEF46
:103830008083CE010E94911BCE010E946D1C6FEF10
:10384000CE010E94711C6E018AE0C80ED11CC60117
:103850000E94181DC6010E94281D5E0188E1A80E65
:10386000B11CC5010E94D41C9EE0E92E0FE020E1AE
:103870004BE06DE0CE01825B9F4F0E94E6218E01FE
:103880000B5D1F4FC8010E94C523C5010E94DE1CAD
:1038900065E0C6010E945F1D811112C0898D8823D9
:1038A00079F040E06EE67BE0C801DF91CF911F9197
:1038B0000F91EF90DF90CF90BF90AF900C94642465
:1038C00060E0C801DF91CF911F910F91EF90DF90E1
:1038D000CF90BF90AF900C947E2621E0FC01208316
:1038E000089570E085E00C94392BAF92BF92CF928F
:1038F000DF92EF92FF920F931F93CF93DF93EC0130
:1039000089819A812FE0289F8001299F100D112421
:1039100085E10E941C2B800F911F24E096958795CE
:103920002A95E1F79A8389832881222391F1AC813A
:10393000AD80B12CC12CD12CE885F9857F0100E048
:1039400010E06E817F819B0140E050E08617970771
:1039500028F0BC01E817F90708F4BF0180E090E007
:103960001F921F921F92AF930E94CB2D6B830F90DB
:103970000F900F900F9070E085E0DF91CF911F9135
:103980000F91FF90EF90DF90CF90BF90AF900C948D
:10399000392BDF91CF911F910F91FF90EF90DF9026
:1039A000CF90BF90AF900895FC018CE39FE093838C
:1039B000828384E0818381E084870895CF93DF93BD
:1039C000EC018C819D81892B81F18C858F7151F562
:1039D00084E10E941C2BBC01882777FD8095982FDD
:1039E0000E94512E26EE3FE34EEC50E40E94DD2E65
:1039F0000E94232E9B017B836A836115710581F0F0
:103A000084E08983FE0140E084819581281739078D
:103A100010F449830AC04F5F32964430A9F702C0C0
:103A20008FEF89838C858F5F8C87DF91CF9108958D
:103A3000FC0188E0808389E0818387E0828386E0DF
:103A4000838384E0848382E0858381E18683089593
:103A5000DF92EF92FF920F931F93CF93DF937C013E
:103A6000EC0100E010E0DD24DA9462E088810E943D
:103A7000C12B88810E94302CF701E00FF11F892BA8
:103A800021F487818F5F878308C08781882349F06D
:103A90008F3F11F4178201C0D78260E088810E94B5
:103AA000C12B0F5F1F4F219607301105F1F6DF91F3
:103AB000CF911F910F91FF90EF90DF900895FC013F
:103AC000E60FF11D81E09781913009F080E00895C3
:103AD000860F911DFC01278130E050E04F5F5F4F62
:103AE00081E02417350709F080E00895262F30E0A3
:103AF000FC01E20FF31F8781423028F481508E3F92
:103B000048F080E008958F3FE1F3642F0E94502F2A
:103B10009130B9F781E008958EBD00000DB407FE25
:103B2000FDCF8EB50895DC01643508F053C04033F5
:103B300008F050C090968C919097342F359535951C
:103B40003595E62FFF27E7FDF095242F277082306B
:103B500099F4DF01A158BC4F84E53802A00DB11DD6
:103B600011248C9190E0022E02C0959587950A94BD
:103B7000E2F78095817009C0833039F446271C969E
:103B80008C91482740FF03C014C0811112C084E506
:103B90003802E00DF11D1124E158FC4F81E090E066
:103BA000022E01C0880F0A94EAF78095908198232D
:103BB00010C084E53802E00DF11D1124E158FC4FDE
:103BC00081E090E0022E01C0880F0A94EAF790810C
:103BD000982B908308951F93CF93DF93EC01162FBA
:103BE000F89460E08F850E94FA2B888918161CF4DF
:103BF00060E00E94FA2B812F0E948C1D8889181684
:103C00001CF461E00E94FA2B7894DF91CF911F9110
:103C1000089528EF31E0EFE7F3E0DF01A9011D92FD
:103C200041505040E1F7DC0119961C9219971A9601
:103C30001C920895DF92EF92FF920F931F93CF9300
:103C4000DF93EC018C858F5F8C878FE7E82E83E014
:103C5000F82ED12C6D2D6064CE010E94EB1D60E822
:103C6000CE010E94EB1D61E08F850E94FA2B8889AE
:103C700018161CF460E00E94FA2B00E010E0F70137
:103C8000E00FF11F80810E948C1D0F5F1F4F0435D4
:103C90001105A9F7888918161CF461E00E94FA2B17
:103CA000D39484E5E80EF11C86E0D812D3CF60E40B
:103CB000CE01DF91CF911F910F91FF90EF90DF9098
:103CC0000C94EB1DFC0160A361A30895FC0160A3AB
:103CD00041A30895CF92DF92FF920F931F93CF934A
:103CE000DF931F92CDB7DEB76C01062FF42E10E0E4
:103CF000121754F4412F4F0D602FC60129830E94E3
:103D0000931D1F5F2981F4CF0F90DF91CF911F91F9
:103D10000F91FF90DF90CF900895CF92DF92FF92A6
:103D20000F931F93CF93DF931F92CDB7DEB76C0134
:103D3000062FF42E10E0121754F4612F600F4F2D50
:103D4000C60129830E94931D1F5F2981F4CF0F9024
:103D5000DF91CF911F910F91FF90DF90CF90089549
:103D6000EF92FF920F931F93CF93DF93EC01F62E08
:103D7000142FE22E0E948D1E4FEF400F410F2E2D6B
:103D80006F2DCE010E948D1E202F412F6F2DCE0151
:103D90000E946A1E6FEF6E0D6F0D202F412FCE0116
:103DA000DF91CF911F910F91FF90EF900C946A1EBD
:103DB000DF92EF92FF920F931F93CF93DF93EC016B
:103DC000E62ED22EF42E112707FD1095040F111D9B
:103DD00047FD1A958F2D992787FD9095801791079C
:103DE00044F42D2D4F2D6E2DCE010E948D1EF39487
:103DF000F1CFDF91CF911F910F91FF90EF90DF9066
:103E000008958F929F92AF92BF92CF92DF92EF92DE
:103E1000FF920F931F93CF93DF93EC01E62ED42EE6
:103E2000122FCC24C394C21AB22EB194BB0CF12C25
:103E3000802F8470A82E802F8270982E802F8870FB
:103E4000882E0170F1160CF04DC0C7FC04C0115053
:103E5000B394B394CB0CF3948F2D880F8F5FC80E5F
:103E6000AA2071F0412F4D0D6F2D6E0DCE010E94D5
:103E7000931D4F2D4D0D612F6E0DCE010E94931D90
